:020000000428D2
:08000800831600308100003076
:100010008B008316F1308500F6308600811783123D
:1000200003018500860086158515FA308C007F2037
:1000300085110C308E004A20C8308C007F206E2045
:1000400032308C007F2008308E004A2032308C0005
:100050007F20752008308E004A2032308C007F20AF
:1000600001308E004A2032308C007F2065203230F3
:100070008C007F2008308E004A2032308C007F2098
:10008000752032308C007F2003308E004A206E2095
:10009000861149280515AF308C007F2006140F30DB
:1000A0008C007F200610AF308C007F20051132308D
:1000B0008C007F2085147D308C007F2085103230AD
:1000C0008C007F208E0B4A2808000614FA308C0022
:1000D0007F203C308C007F2006100800652006142D
:1000E0007D308C007F200610080065200614FA3051
:1000F0008C007F2046308C007F2006100800643082
:100100008D0085208C0B7F28080000000000000077
:0E01100000000000000000008D0B8528080094
:00000001FF
